:040000006F30102924
:100004000000000000000000BA370000DA370000EA
:10001400000000008E3A0000000000000000000014
:100024008E3A00008E3A000000000000000000003C
:100034008C2F00000000000090020000000000006F
:100044008E3A00008E3A00008E3A00008E3A00008C
:100054008E3A00008E3A000082330000AA3300007A
:10006400D2330000FA330000223400008E3A00003C
:100074008E3A00008E3A00008E3A00008E3A00005C
:100084008E3A00008E3A00008E3A00008E3A00004C
:100094008E3A00008E3A00008E3A00004A34000086
:1000A4008E3A00008E3A00008E3A00008E3A00002C
:1000B4008E3A00008E3A00008E3A00008E3A00001C
:1000C4008E3A00008E3A00008E3A00008E3A00000C
:1000D4008E3A0000703700008E3A0000B8400000ED
:1000E400C23400008E3A00008E3A00008E3A0000BE
:1000F4008E3A00008E3A00008E3A00008E3A0000DC
:10010400000000008E3A00008E3A00008E3A000093
:100114008E3A00008E3A00008E3A00008E3A0000BB
:100124008E3A00008E3A00008E3A00008E3A0000AB
:100134008E3A00008E3A00008E3A00008E3A00009B
:100144008E3A00008E3A00008E3A00008E3A00008B
:100154008E3A00008E3A00008E3A00008E3A00007B
:100164008E3A00008E3A00008E3A00008E3A00006B
:100174008E3A00008E3A00008E3A00008E3A00005B
:100184008E3A00008E3A00008E3A00008E3A00004B
:100194008E3A00008E3A00008E3A00008E3A00003B
:1001A400000000000000000000000000000000004B
:0C01B4000000000000000000000000003F
:1001C00097020120938202E4938202E0739002344A
:1001D00003210500224573100530B1A819712320B1
:1001E000250006C006C216CAF322003093F2820030
:1001F000638402009302000816C412C81ACC1ECEF3
:1002000022D026D22AD42ED632D836DA3ADC3EDEB6
:10021000C2C0C6C2CAC4CEC6D2C8D6CADACCDECE26
:10022000E2D0E6D2EAD4EED6F2D8F6DAFADCFEDE96
:1002300003A1050009A002457310153492403785CB
:10024000000013050580732005302245732005301A
:100250004242D2426243F243025492542255B25572
:100260004256D2566257F257064896482649B64932
:10027000464AD64A664BF64B065C965C265DB65DF2
:10028000465ED65E665FF65F09617300203000004F
:10029000197116CA9302000816C49302000273A0D3
:1002A000428006C212C81ACC1ECE22D026D22AD430
:1002B0002ED632D836DA3ADC3EDEC2C0C6C2CAC456
:1002C000CEC6D2C8D6CADACCDECEE2D0E6D2EAD4E6
:1002D000EED6F2D8F6DAFADCFEDE73110134EF0066
:1002E0008061EF103009EF00C06373110134138493
:1002F0008189032904006304090223200400732573
:1003000010342AC013840189044023A024001384DC
:100310004189044003A10400024573101534924042
:10032000B78200009382028073A00230A24273A0C1
:1003300002304242D2426243F24302549254225566
:10034000B2554256D2566257F25706489648264949
:10035000B649464AD64A664BF64B065C965C265D25
:10036000B65D465ED65E665FF65F0961730020305B
:100370000000397101436EC619A0397141536AC832
:1003800066CA62CC5ECE19A0397101535AD056D2DA
:1003900052D44ED64AD826DA22DC06DE330161403A
:1003A000828241114AC026C222C406C68282B24D50
:1003B0004101024D924C224CB24B4101024B924AF8
:1003C000224AB2494101024992442244B2404101C9
:1003D00082803D432A876373C3029377F700BDEFA2
:1003E000ADE5937606FF3D8ABA960CC34CC30CC7A5
:1003F0004CC74107E36BD7FE11E28280B306C340CE
:100400008A069702000096966780A6002307B70029
:10041000A306B7002306B700A305B7002305B7005E
:10042000A304B7002304B700A303B7002303B70056
:10043000A302B7002302B700A301B7002301B7004E
:10044000A300B7002300B700828093F5F50F9396C1
:100450008500D58D93960501D58D61B793962700BC
:100460009702000096968682E78086FA9680C117EA
:100470001D8F3E96E374C3F8A5B703A581808280E3
:10048000EFF23FF2938781809843050798C3EF10FE
:10049000C0313C45FD173CC589E77C413CC5EF10A8
:1004A0008035EF10806005B7634205029307803EF8
:1004B0003347F5023365F5023305F5021305753E42
:1004C0003345F5023307F7023A9582807D558280E5
:1004D00001458280014582800145828001458280FC
:1004E000EFF23FEC19649964130404BD9384C4BD16
:1004F00063639400C9BD1C4011048297D5BFEFF21D
:100500005FEA196499641304C4BD938444BE6363B1
:10051000940055BD1C4011048297D5BFEFF27FE8CF
:10052000F93FEF30802D45B5EFF2BFE7B70500008A
:1005300037450000D14715479306002001469385B3
:10054000C55113058558EF10A026EF10203EA5BD1C
:10055000EFF23FE5EF10E062EF20F01BEF00B02B71
:10056000EF10205CEF005078C137EF10205C012CB9
:10057000EF00707A014581BDEFF2BFE2D13F014546
:1005800099B5EFF27FE0AA89EF10202219C1EF1090
:10059000800A2545EF00F06044411304450063964E
:1005A0008400EF108020014911A8138944FF2146DF
:1005B000CE854A851D2D01E9EF10201F19C1EF10CE
:1005C000E0084A85E5BB8440D9BF09E57D558280B6
:1005D0007D55D5BBEFF2FFDC2A842E853289AE84AF
:1005E0004D377DF522852686A545EF00305E014515
:1005F000231C2401230E0400231D0400D9BFEFF2A5
:100600005FDA1E2D41112A84C18B9DE71C558DC3D5
:100610002EC68297AA84B24501CD2A8637450000AE
:10062000A28513050559EF0090182685410161BB8D
:100630001E2C93E707011EAC1E2CA18B89C73E2CF4
:10064000E554A18BFDF35C5489CF22858297AA845F
:1006500005E13E2C93E787003EAC5C2C85075CAC43
:10066000E9B785679387F7F0FD8D2EAC8144D5B748
:10067000E957E31CF5FAF1BF5C2D85CBEFF27FD291
:10068000FD1793F7F70F5CAD2A84014789EF1C59DA
:1006900089E70147231D040039A082972A8775D96D
:1006A000E957E309F5FE3A8539BB7D573A858280E3
:1006B000EFF23FCF582D09E77D552129014521A0B3
:1006C0005C5999C3829701B36955C5BFEFF27FCDDD
:1006D000582D09E77D55F52E014521A01C5D99C3D4
:1006E0008297D5B16955C5BF0CD101458280EFF223
:1006F000BFC993894186854A83A7418663863705AA
:10070000EF10204883A741862A8A638D370303A40C
:1007100041865C4018401309C4FE5CC398C340C0C6
:1007200000C0EF0050717C5099C34A8582974A857A
:10073000EF00105B631B55014A85EF00104FEF007F
:10074000F0705285EF10A04495B9EF0030705285DB
:10075000EF10E0434848EF00303A4A85EF0030554B
:1007600061BFEFF21FC413848193130904011C407D
:1007700091C382971104E31C24FF953FEDB7EFF27C
:100780005FC237060000B7450000930800023D48ED
:10079000930700201387819481461306267693855C
:1007A000855C1385818BEF00307D1385818BEF1085
:1007B000E01711B9EFF2FFBE41112A842E8532C62F
:1007C0002EC4EF1060083246A24519C68547630D56
:1007D000F60001454101C5BE5840938745011CC341
:1007E00098CD5CC0C0C9F5B71C406388870083C63C
:1007F000550303C7170263FAE600D4431387450184
:1008000098C294CDD8C3DCC9E9B79C43F9BFEFF2D5
:100810005FB94111B2842E8689452A8436C6EF001D
:10082000F03AB246930744011CCC5CC846AC14B401
:100830000145410149BEEFF23FB583A70185411152
:100840002EC62A8491C38297EF10A0335E2CAA890A
:1008500089CFFD175EACEF10803383A7C1840145BB
:1008600091CB22858297014531A0B24791E7EF10E5
:1008700000327955410199B6EF0030732328050203
:100880001034AA85AA84130544012D37B247635C4E
:10089000F0001389C404700081454A85EF10601D83
:1008A0004A85EF1000124E85EF10602EEF00704960
:1008B000885845D5C1B7EFF2DFAE83A781842A847B
:1008C00091C38297EF10E02BAA8448489307440114
:1008D000630EF5003115EF10A00005442685EF10DA
:1008E000002B19C0EF00F0450145F1BC5E2C8507D7
:1008F0005EAC0144E5B7EFF2DFAA4111EF106028CA
:10090000138741811C23850793F7F70F1CA383A747
:10091000C18081C72AC682973245EF104027410126
:100920005DB4EFF21FA84111EF10A025138741819C
:100930001C23FD1793F7F70F1CA383A7018181C721
:100940002AC682973245EF1080244101ADBC03C511
:1009500041818280937808044111639E0800916868
:100960009388487793730801638B03001378E8FF3B
:10097000930E000219A891689388086DE5B7137368
:100980001800930E0003E30503FE13732800630EA3
:100990000306635806023306C0409302D0020A8E53
:1009A000814F294F6395E6073373D6023356D6023B
:1009B000469303430300850F050EA30F6EFE7DF2E1
:1009C0000DA0137348009302B002631703009372E3
:1009D0008800B3325000960279F2930600035480E7
:1009E000854FFE8663D3FF00BE8613781801158FEE
:1009F00063130804638502006353E0007D172A86B1
:100A0000B308E5001303000221A88142F1B7137374
:100A1000F600118271BF6374B600230066000506FC
:100A20003388C840E34900FF3A8663530700014614
:100A30007D173295118F638802006374B50023001F
:100A400055007D17050563870302AA961308000366
:100A50001DA86374B6002300D60105063388C8407C
:100A6000E34900FF3A866353070001467D1732953C
:100A7000118FE1BF2A86B308E500CDB76374B500D6
:100A80002300050105053386A640E3C9CFFEFD56C8
:100A9000FD1F6383DF0099E7AA873306E50013088B
:100AA000000231A86376B5003306F101102210A1CF
:100AB0000505F9BF63F4B700238007018507B30676
:100AC000F640E349D0FE6353070001473A954101E0
:100AD0008280EFF21F8D2A849D3D09C523AC818061
:100AE0006FF07F8EEF00704C75D900D9D5BF0D47E0
:100AF000AA876376C7009377350091C7AA873E9689
:100B00006397C706828093F7F50F13978700D98FF5
:100B1000139707015D8FB308C500AA87BD463388C8
:100B2000F84063EB060393574600C156B386D702DD
:100B30009207AA970D4836963383C700BE86B3083E
:100B4000D3406362180313572600F156B306D70249
:100B50000A07BA97369665B798C3D8C398C7C1072E
:100B600023AEE7FE6DBF910623AEE6FEC9BF850743
:100B7000A38FB7FE71B763F2A504B386C500637E89
:100B8000D5029345F6FF8147FD176393F5008280F8
:100B90003387F600030807003387C7002A9723002E
:100BA0000701DDB73387F500830607003307F5003B
:100BB000850714A3E318F6FE82808147E5BF0DC6C2
:100BC000AA8785050387F5FF85079306F6FFA38FA0
:100BD000E7FE09EB3E9685076393C7008280A38FEB
:100BE00007FED5BF3686F1FE828001476314E6001A
:100BF000814739A8B307E50083860700B387E5007E
:100C00009C23B387F640E207E18799E30507F9FEE5
:100C10003E858280AA870387070001E73385A740C6
:100C200082808507CDBFEFF24FF52E89B30B2501EA
:100C300041112A8CB68563F5AB001349F5FFFD5BC6
:100C4000C169374A00006284930AB002130B0002A4
:100C5000FD19130ACA7631A8130750026389E70207
:100C6000637374011CA013051400B284138614006E
:100C70002A8483070600EDF363060900637B742F63
:100C8000230004003305844141016FF08FF20148D5
:100C90001307D002930630021305000331A0639EB0
:100CA0005701136848002686830716009304160030
:100CB000E397E7FE13680801FDB7639567011368C2
:100CC0008800D5B76395D70013680802E9BF63951C
:100CD000A70013681800C1BF138707FDA54663E688
:100CE000E6040147A546294539A03307A702850434
:100CF0003E97130707FD83870400138607FDE3F67D
:100D0000C6FE038604009306E002FD57631FD60467
:100D100083871400254693861400138507FD6365B9
:100D2000A60A8147254529433DA09306A0027D5789
:100D3000E399D7FC9841930426009105E35307FCFF
:100D40003307E040136808016DBFB387670285066B
:100D5000B297938707FD03860600930806FDE376A6
:100D600015FF63D307008147B6848386040013060A
:100D70008006014593F8B6FF6395C80013F5F60F9A
:100D8000850403860400930690066303D60663C5B4
:100D9000C606930680056303D61C63C3C604930787
:100DA00050026307F61A63757401930750021CA082
:100DB00083870400130514006386071A63737501A3
:100DC0001CB0130524005DB51306A0026397C7008D
:100DD0009C4193862400910569B7B684814771B719
:100DE000930630066302D60893064006E31DD6FA42
:100DF00013682800A94699A0930630076303D60C10
:100E000063C5C6029306F0066300D6169306000774
:100E1000E31BD6F8FD566315D70013681800214769
:100E2000938C4500C14690411DA893065007E303EB
:100E3000D6FC93088007C146E31716F71306C006D1
:100E4000938C4500E301C5FE13068006E31DC5FC37
:100E5000904193752800639B051033763601DE853B
:100E60002285CD3CE68519B5137808016315080283
:100E7000BA879306000229A06373740114A00504C5
:100E8000FD17E34BF0FE9307F7FF6343E0000547D0
:100E90003387E740050793874500637474019441E5
:100EA00014A013051400229713060002B306A740EE
:100EB0006344D000BE855DBB6373750110A1050559
:100EC000F5B783AC0500138D450063930C00D28CFD
:100ED00066853EC63AC442C2353BB247AA8612482E
:100EE00022476355F00063D3A700BE86137808013C
:100EF000631E0800BA871306000231A063737401F1
:100F000010A00504BA877D17E3CAF6FE814763C1C6
:100F1000D702B68763D3060081473305F4002A97CA
:100F200013060002B307A74063CFF600EA853DBB76
:100F30003306F40063777601B385FC0083850500F2
:100F40000CA28507E9B76373750110A10505D9BF28
:100F50006373740110A01305140009BB136808041F
:100F6000C146E9BDFD1419B3A146C9BD420641867B
:100F7000FDB5A38F0BFE39B303A5C1818280EFF2CB
:100F80004FC203A9C181EFF0CFDF11CD1384C1811E
:100F9000AA84084019C1EFF02FEE9305300426858E
:100FA000EFF0EFE504C04A856FF0EFC18280397140
:100FB00026CA2ED232D436D62A8654109305F0078C
:100FC000138581B43EDA36C606CE22CC3AD842DC4E
:100FD00046DE9139AA8603A5C18109E9138581B44A
:100FE000F137F2406244D244216182802686262D68
:100FF0001384C18193E704043EAD9307F00763F4C3
:10100000D7009306F007138681B48145EFF00FEC0B
:101010001C40A6AFF9B7EFF2CFB837450000130573
:10102000456E7137374500001305056F493737475F
:10103000000037450000130747718D4605468D4572
:1010400013050572AD373745000013050574853764
:101050006FF06FB731C591661377F50F9386065D14
:1010600009C7BA96882205058280C167938707F071
:10107000E98F81CB21851377F50F36970823250556
:101080008280B707FF00E98F81CB41859377F50F09
:10109000B6978823450582806181369508216505CC
:1010A000828003A741825C41BA976305F502B623AB
:1010B00095E283A60182638FF60093868182904237
:1010C0006313F60088C2D44354C1DC43B306E54041
:1010D000BA9794C71045B307C700630FF500B6234E
:1010E00081EE938681828C426393A5009CC2544119
:1010F000D4C35C413E9710C78280EFF28FAA83A5CC
:1011000001833745000013058578553583A5C183D4
:10111000374500001305C579593D83A5C182374580
:1011200000001305057B61356FF0EFA9EFF26FA7A3
:1011300013F7C5FFE1462E8663F1E60693073500F7
:10114000F19B930687FE63EAF6041D8F130687FE64
:1011500023A8C1828966511713844182938606EAC7
:10116000D8C394C323A407001CC0BA9723A0F1825C
:10117000C966938606EAB755000094C3D8C398C7DA
:101180008146054693858584138581BCEFF02FE861
:10119000184023A4E1826FF00FA3AA853755000001
:1011A000130505852935C5BFEFF2AF9F39C503A7E4
:1011B00001831304350071981389018381446366A8
:1011C000870EB1476373F4003144FD55138581BC2C
:1011D000EFF06FE683A7818283A54182832809000F
:1011E00026853386B740B38688401388818263683A
:1011F000D600138581BCEFF00FEC81447DA0B38451
:10120000C500BA2003AE440061E73307CE40930F18
:1012100047FF63EF8F0A138FC183938EC18213033D
:10122000840183260F0083A30E001389C183938258
:10123000C18263EF6F061307C4003297896E338350
:10124000E500938E0EEA2322C3012324C30023204A
:10125000D3010546D8C0B2A003264300B1086304F9
:1012600016012E9618C61387C60022972320E90080
:1012700063F4E30023A0E2000967130707EA9AA0DA
:10128000639A970083A601820147B22305EE19C332
:101290002320F800138581BCEFF0EFE183A7818361
:1012A000B10481C7A2852685829726856FF0AF910C
:1012B00005463697B2A02320EF00E3FFE3FA23A010
:1012C000EE005DBFE385D7FCDC430547AE9775BFF5
:1012D000728631BFEFF2EF8C3306B50241113285D1
:1012E00032C6D9352A8409C532468145EFF03F80A0
:1012F000228541016FF02F8D45C5EFF2EF8883A75E
:1013000041832A8491C3829783A7418213894182B2
:101310006366F40883A701826372F408FD551385A0
:1013200081BCEFF04FD1835764FF930944FF81CB19
:10133000035744FF8967938707EA6301F70237453C
:1013400000001305C57FA531835644FF035664FF93
:1013500037550000CE8513058581913989679387BC
:1013600007EA231AF4FE938781829843231B04FE25
:1013700063F4E90023A037011387C1831C4383264C
:1013800084FF4E85958F83260900B386D940B69792
:101390001CC3013B138581BCEFF0EFD16FF00F82CE
:1013A0008280B707002093860700014793870700D4
:1013B00021468C426396A500131547003E95828016
:1013C0000507C106E317C7FE01458280EFE2DFFB98
:1013D0002A842E85AE89328AE9372A89A92C83246A
:1013E0004900930749006390F4048D2493E909F8B8
:1013F000230434012146D2852285EFF04FFC83A7D8
:10140000018499C322858297EF00A07703274900C2
:101410009307C4005CC358C42322F90004C8EF003A
:1014200000776FE0BFF984407DBFEFE29FF783A7AD
:1014300041842A8491C3829723040400EF006074DE
:10144000544418489307C400D8C214C31CC85CC4D1
:10145000EF00E0736FE03FF7EFE21FF32E89AA89F8
:101460008937AA84484589332A841DCDD0448145D3
:10147000EFF0EFE7214623043401A3040400CA85FA
:101480002285EFF0CFF383A7018499C32285829749
:10149000EF00206FD8409307C40091045CC358C488
:1014A0009CC004C8EF00A06E22856FE03FF1EFE220
:1014B0005FEF83A741842A8491C3829723040400A9
:1014C000EF00206C544418489307C400D8C214C3DA
:1014D0001CC85CC4EF00A06B2285393D6FE0BFEEF5
:1014E000030585007D81828023900186938781BEDC
:1014F00013870708DCC39CC3A107E39DE7FE3D47B4
:10150000238AE18423AC018423A601869387418644
:10151000DCC39CC38280EFE2DFE803A5C186EFF065
:101520007FB37D1593173500138581BE3E95084125
:101530001307C5FE210523ACE184EFE07FC86FE00F
:101540009FE8EFE21FE6EF00C063839701862A89D8
:10155000B1E703A5C186EFF0FFAF7D151317350086
:10156000938781BEBA97844393878185804393850F
:10157000C4FE6305B4028CC383A7C185238AA184FA
:1015800099C32285829783C741811305C40193853E
:10159000840093F7F70F81EBEFE05FC44A85EF001B
:1015A000005F6FE05FE2EF00E05ECDBFEFE27FDF64
:1015B0002A84EF00005D8347440393064401C19BE6
:1015C00093E71700230AF402834754031397370065
:1015D000938781BEBA97D84314C318CCD4C35CC8D0
:1015E0009387C1869443185C558F98C3EF00205AA7
:1015F0006FE07FDDEFE2FFDA2A846123184C544864
:1016000093074401D8C214C35CC81CCC834754035D
:1016100013973700938781BEBA979843631AF700F0
:101620001387C1861C5C144393C7F7FFF58F1CC357
:10163000B92B6FE05FD9EFE2DFD6A1239387018654
:101640009A2305079AA3A1236FE0FFD7EFE27FD586
:101650000D2B138701861E23FD17C207C1871EA30A
:10166000634BF000231007001D2383A7818591C3DE
:10167000C93D6FE05FD5212BEDBFEFE29FD203A400
:1016800081850123AA842285B5379147230AF40274
:101690001305C404012E2285A1358547631BF5007F
:1016A0003C5C81EB228551332685D521593D6FE085
:1016B0009FD183A641861307440123A2E186D8C2A5
:1016C0009387418654C81CCCC5B7EFE29FCD2A84CE
:1016D0005105411108CC48C80CD050D014D43A86DA
:1016E00058D49305300236853EC642C4EFF02FC071
:1016F000585410544C5008507117B71600003A96C1
:101700009386A6672D21B24722483716000048CCA1
:10171000230BF402A30AF402232C040281472322A0
:1017200004052324040523280402230A0402232C8D
:101730000406232E04060147A28613068675A28599
:101740001305C4041D2483A7018799C322858297AA
:10175000014541016FE03FC7EFE2BFC45049144D5E
:10176000795718D954C21307450190C218CD58C9EA
:10177000353DC13B6FE03FC5EFE2BFC24111B284CE
:101780002E8685452A84368946C03AC63EC442C262
:10179000EFF0DFC3024892472247B2464A86A68549
:1017A0002285253741016FE01FC203A58185828014
:1017B000EFE29FBD41112E89AA85054532C6B68448
:1017C000BA893E8AEFF05FC92A8411C92685EFF0F5
:1017D000BF9D324609E92285EFF07FCD0144228585
:1017E00041016FE0BFBDAA865288CE872687CA8591
:1017F0002285E13DEDB7EFE2DFBA612683A781855F
:101800000546AA8603C747033D8B631CC702D04B1E
:10181000984F6308E60258C210C303C65703938665
:1018200047010E06138781BE94CF3297504314C2EE
:1018300090CF54C3D8CBA12EEFF0BFD001456FE0BD
:101840009FB83685A926DDBF834745030547BD8B75
:10185000639FE702EFE2FFB42A842526834744030F
:10186000AA842285C19B93E72700230AF402EFF0A4
:101870007FD81305C404F1222685112E83A7818702
:10188000014581C72285829701456FE0DFB37D5511
:101890008280EFE21FB141112AC6E52403A48185AD
:1018A0002A89228555379304C40470008145268512
:1018B000C922268539224A85D92CEFF09FC81858AD
:1018C000F9576314F70023280402014541016FE032
:1018D0009FAFEFE21FADEFE03FBD653F6FE0BFAEF2
:1018E000834745030947BD8B6390E704EFE27FAB75
:1018F0002A84412C5448184C93074401AA84D8C226
:1019000014C31CCC5CC81305C404252A26854124B5
:101910002285EFF0BFC983A74187014581C7228592
:10192000829701456FE03FAA7D558280EFE27FA755
:101930008346650305473317D70018DD0947A30A17
:10194000D502230AE502693F83A7818599C3EFF099
:101950005FBF01456FE03FA75449184D930745010C
:10196000D8C214C31CCD5CC98280EFE29FA3411191
:10197000B2842E86A9452A8436C63AC43EC2EFF008
:10198000FFA49247B2462247F99B1CB49307440137
:1019900044CC14D02324040258D01CCC5CC8410190
:1019A0006FE07FA2EFE2FF9F2A84E12AAA842285CA
:1019B00065372685E92A2285EFF03FA701456FE0CC
:1019C0009FA0EFE21F9E2A846D2AAA842285693790
:1019D0001C342685F99B1CB45D2A83A7C18499C356
:1019E00022858297EFE07FA95C503E9508D4512A6A
:1019F00013878188032847003706008093878188F2
:101A00001346E6FF98436315F8029386C187904218
:101A1000050690C29306440154C358C894C31CCC15
:101A20001C3493E717001CB49D2201456FE0BF9959
:101A3000544B0C546385B6008D8EE378D6FCBA8780
:101A4000D1B71C35858B85C7EFE2BF9583A781840D
:101A50002A8491C382973522AA842285F53D268562
:101A60003D221C340145F99B1CB46FE0DF957D5588
:101A7000828085476381F50263C5B70085C1014552
:101A800082808947638FF5008D47E39AF5FE1C3508
:101A900093E7270009A85C511CC2D5B71C425CD152
:101AA000F9BF1C35F59B1CB5D9BFEFE21F8DEFE0E8
:101AB000DF9C2A8CF920B70900802A8A93848188C8
:101AC00093C9E9FF8D4B8040631694005285C12075
:101AD0006FE03F8E48481309C4FE3305AC40E3E78E
:101AE000A9FE83A7018899C34A8582974A85EFF0AA
:101AF000BFE61C4448448297EFE03F9883A74188A3
:101B00002A8C99C34A858297834754FF13F7E70FBE
:101B1000A30AE4FE8D8BE39877FB4A85EFF07FEA1A
:101B20005DB793878188DCC39CC382808280110665
:101B3000719A2A8837C7ADDE130506F8AA871307FE
:101B4000F7EE631EF600A167938707882322D6F875
:101B50002324B6FA232006F92324F6F8828098C3BA
:101B60009107C5B737F700E01C43B7060080D58F53
:101B70001CC3828037F700E01C43860785831CC3A3
:101B800082802165130505807315053082807310EE
:101B900005308280EFE2FF801387818918439387A5
:101BA000818919E323A8A18823AAB188054798C38E
:101BB000553F6FE05F812A87814718436314A70070
:101BC0003E8582808507D5BFB707EFBE37E700E0C7
:101BD000938707083CC701458280EFE28FFC3755A9
:101BE00000001305C588EFF08FBC01456FE0AFFD25
:101BF000EFE22FFB2A84FD54375900007D14631453
:101C000094006FE04FFC130549FFEFF04FBAFDB7AA
:101C1000EFE28FF70041AA8437590000B75900005E
:101C2000631494006FE08FF99305C4FE130589FFD8
:101C3000EFF0EFB71C40638697001385C9FFEFF004
:101C40000FB70040F1BFEFE2CFF52E89EFE09FFC28
:101C50002A84EFF05F9E83240900639C2401EFF047
:101C6000FF9EA14763C3870011E0214422856FE0F6
:101C70008FF5138544FFEFE0FFF96353A4002A8436
:101C80008440E1BFEFE26FEF0545EFF08FF1B75908
:101C90000000130945002A84CA85138509B46537F5
:101CA000AA85AA8437550000138609B4130585B4A4
:101CB000EFF0EFAF2685EFF0BFF3375500001305C7
:101CC000C5B8EFF0CFAE4040B7590000054A894A89
:101CD000375B0000B75B0000375C0000B75C0000BA
:101CE000375D00006315890001456FE08FEC034705
:101CF00094021385C9BC930644FF2146A685EFF0E4
:101D00000FAB8347840213858CBDBD8B638E470167
:101D100013054CBE638A570113850BBF91C711474A
:101D20006396E7001305CBBFEFF06FA84C4C930709
:101D30003002AE8698226306F702105093074006E1
:101D40000848B295B386D540B386F602585C5C501D
:101D5000898D13058DC0B3D6C602EFF04FA50040A4
:101D600051B78506C1BFEFE22FE241110945EFF0FF
:101D70004FE393094500375900002A84CE851305A7
:101D800009AEEFF05FECAA85AA8437550000130670
:101D900009AE1305C5AEEFF08FA12685EFF05FE524
:101DA00037550000130585B0EFF06FA04040375A5B
:101DB0000000B75A0000376B0000639689000145A8
:101DC00041016FE0AFDF1A281C44930644FF13095A
:101DD000840036C63AC44A856306F902EFF0BFDDD7
:101DE0002247B246AA872146A68513850AB2EFF09C
:101DF0000F9C4A85EFF0DFE113058BA5EFF02F9BD9
:101E0000004065BFEFF03FDB2247B246AA8721467C
:101E1000A68513050AB3EFF08F99DDB7EFE2CFD6B1
:101E200041111145EFF0EFD79309450037590000F4
:101E30002A84CE8513054992EFF0FFE0AA85AA8493
:101E400037550000130649921305C592EFF02F96FF
:101E50002685EFF0FFD93755000013050595EFF003
:101E60000F954040375A0000B75A0000376B00000A
:101E700063968900014541016FE04FD41C4413096A
:101E80008400930644FF18486309F9024A8536C660
:101E90003AC4EFF05FD22247B246AA872146A68510
:101EA00013850A97EFF0AF904A85EFF07FD61305C0
:101EB0008BA5EFF0CF8F004065BF2146A6851305A7
:101EC0008A98EFF0CF8EC5BFEFE20FCC41110D45E0
:101ED000EFF02FCDB7590000130945002A84CA85B9
:101EE0001385C9A7EFF03FD6AA85AA84375500000D
:101EF0001386C9A7130545A8EFF06F8B2685EFF071
:101F00003FCF37550000130585AAEFF04F8A4040B8
:101F1000B759000063168900014541016FE00FCAFF
:101F2000930644FF1305840036C6EFF0DFC803486C
:101F300034015C48B246AA8821472146A68513850C
:101F400089ACEFF0CF860040F1B7EFE2EFC341116B
:101F50001545EFF00FC593094500375900002A8455
:101F6000CE851305C999EFF01FCEAA85AA843755EF
:101F700000001306C9991305459AEFF04F83268593
:101F8000EFF01FC7375500001305859CEFF02F8237
:101F90004040375A0000B75A0000376B0000639684
:101FA0008900014541016FE06FC17A285E28104425
:101FB000930644FF1309840036C63AC43EC24A85DC
:101FC0006307C902EFF03FBF92472247B2462A8813
:101FD0002146A68513854A9EEFE07FFD4A85EFF0F6
:101FE0003FC313058BA5EFE09FFC00404DBFEFF012
:101FF0009FBC92472247B2462A882146A6851305F0
:10200000CA9FEFE0DFFAD5B7EFE20FB841111945EB
:10201000EFF02FB993094500375900002A84CE8587
:10202000130549A1EFF03FC2AA85AA8437550000E5
:10203000130649A1130505A2EFE07FF72685EFF00F
:102040003FBB375500001305C5A3EFE05FF64040E6
:10205000375A0000B75A0000376B000063968900BA
:10206000014541016FE08FB51A2C1C44930644FFD3
:102070001309840036C63AC44A856306F902EFF0B4
:102080009FB32247B246AA872146A68513854AA553
:10209000EFE0FFF14A85EFF0BFB713058BA5EFE046
:1020A0001FF1004065BFEFF01FB12247B246AA877B
:1020B0002146A68513058AA6EFE07FEFDDB7EFE2A4
:1020C000AFAC5D712545EFF0CFAD9165130600050E
:1020D0002A8413094500938585530A85EF2020340F
:1020E000B7590000CA851385C98BEFF0DFB5AA8503
:1020F000AA84375500001386C98B1305458CEFE081
:102100001FEB2685EFF0DFAE375500001305C58EB7
:10211000EFE0FFE94040D149375A000063168900DB
:10212000014561616FE08FA91C44930644FF63E0A1
:10213000F90298088A07BA9703A707FB1C282146CB
:10214000A68513050A91EFE09FE60040C1BF464710
:10215000F5B7EFE26FA32945EFF0AFA4B759000040
:10216000130945002A84CA85138509C3EFF0BFAD62
:10217000AA85AA8437550000138609C3130585C3B1
:10218000EFE0FFE22685EFF0BFA63755000013050C
:1021900005C6EFE0DFE14040B7590000375A0000C4
:1021A000B75A0000631E8900EFE02FADAA853755AE
:1021B0000000130585CBEFE09FDF01456FE00FA026
:1021C0005C4C184C138549C8930644FF2146A685EC
:1021D000EFE0FFDD8347D4FF1385CAC9858B99E300
:1021E00013058ACAEFE0BFDC00406DBFEFE2CF9974
:1021F0003755000013054589EFE07FDB03A4018A12
:10220000B7590000375A000083A7418A6365F4007C
:1022100001456FE0AF9A044009469385898A268577
:10222000EF20002F19C55040A6851305CA8AEFE09C
:102230001FD83104D1BFEFE22F95375500001305A9
:102240008515EFE0DFD603A4018AB7590000375A9D
:10225000000083A7418A636BF40037650000130513
:1022600085A5EFE0DFD401456FE04F9504401946A6
:10227000938549172685EF20A02901E950409385D1
:1022800064001305CA17EFE09FD23104D9B70545A2
:102290008280EFE26F8F79712A84AA9593060002FB
:1022A000254783070400B38485406385D70A638389
:1022B000E70A0145638B0410014913070002A54694
:1022C000B307240183870700638AE7086388D70878
:1022D0006314990883A9018A83AA418A375B0000A5
:1022E00063F0590903AA0900194693054B17528553
:1022F000EF20002259E54A86A28513056A00EF20E7
:10230000202141E14A9A83076A00A5EF83A9890049
:10231000638809041306800281452800EFE06F8B73
:1023200013098100CA86A2870145014713080002EC
:10233000A548294313062002130EC0058385070014
:102340006384050163961505631F9702A94763031C
:10235000F50469A80504B1B705099DB7E31C09F6A2
:10236000A287038707001377F7FD79E73755000049
:102370001305051423800700A285EFE05FC37D5598
:10238000A9A0B109B1BF23800700050785077DB764
:1023900063106504375500001305C511EFE03FC118
:1023A0000018B7540000832509001385C4131109D0
:1023B000EFE0FFBFE31989FE37650000130585A52F
:1023C000EFE0FFBE29452C00829945616FD01FFFC9
:1023D000637E970005056392C504850705079CC2C7
:1023E000838507006381C5026364970069FD8DBF23
:1023F000838E17006396C5016394CE008507050799
:1024000085070507F1BFE37397FE238007000507E3
:1024100085079106E36497F2D1BF9CC283850700CC
:102420006389050163871501E30297FC85070507AA
:10243000F5B7E36097FE5DBF850725B7EFD2FFF3E1
:102440008307050099E781450145EFF0DFDE6FD096
:102450005FF603AA018AAA8981440149375B00001B
:10246000B75B000083A7418A6369FA00EDD04A8612
:10247000A6854E85EFE0AFF4D9BF03240A001946C4
:1024800093054B172285EF20A00821E14E85EF2010
:10249000000719042A86A2854E85EF20600715E5FE
:1024A000631709002285EF2080052A89A284A68768
:1024B00022870386070001EE858F63D327013E89BB
:1024C000A28513854B18EFE09FAE310A61BF8306EA
:1024D0000700FDD2E312D6FE85070507D9BFEFD26C
:1024E0005FECEFF02FFA01456FD0FFEDEFD27FEBFD
:1024F000EFE0BFC001456FD01FEDEFD29FEA03A50B
:10250000C189EFE04FBB01456FD0FFEBEFD27FE910
:10251000B76700009387C7A723A0F18AB7670000B9
:102520009387C7BC23A2F18AB76700009387C7BC13
:1025300023A4F18AB76700009387C7BC93050021E5
:10254000054523A6F18A1384C189EFE0BFD808C0EE
:1025500019E93755000013058523EFE05FA57D5489
:1025600022856FD05FE6B725000037550000A947E8
:102570002D479306004001469385C5681305052540
:10258000EFF00FA3AA840840B7550000814601462A
:1025900093858525EFE0AFA70144F9D02685EFF0BC
:1025A000EFB87DBFEFD2FFDFEFF07FCE0DC5B7559F
:1025B000000093854520138581C6EF105073B755F1
:1025C000000093854521138581C6EF107070138537
:1025D00081C66FD05FDFB75500009385C520E1BF8E
:1025E000EFD23FDC2A843755000013054527EFE082
:1025F0001F9CEFF03FFBAA85375500001306A41B74
:102600001305C527EFE0BF9A01456FD0DFDBEFD29E
:102610005FD941112AC6EFD0DFF6B24511E937552F
:10262000000013058521EFE09F9841016FD0BFD9CD
:1026300083A7C189AA841384C18983A7C720E3869D
:10264000A7FE93053014EFD09FFB65F11C4003A556
:10265000C72009C9EFE04F821C40814503A5C72070
:10266000EFE08F8800401306000581451305A41B89
:10267000EFD03FD6B7250000231504202326942051
:102680009385A54F2685EFE02F8645B7EFD27FCE05
:1026900083A7C18941119384C18903C74702136786
:1026A00017002382E70283A7C72091E7EFE0DF8CC2
:1026B00019C1EFF0DFF5EFF0FFEEEFE05F8F375B72
:1026C0000000B75B0000B7590000376A0000B75A36
:1026D0000000375C0000B75C00009C408546130694
:1026E000F10003A5C720FD55EFD09FFC8547631A75
:1026F000F5000309F100ED4780406319F90008D0A7
:10270000E9BF8840FD55EFE00F93C1BF1C506392B5
:10271000A7029307B0056315F90089471CD075BF60
:1027200023200402E30B09FAA5476314F9120149B7
:10273000D1A80947E398E7FE232004029307100479
:102740006312F9046E30D1D9FD15C205C1816EB096
:102750009307A41B13070005B385E50213060005C4
:102760003E859385A502A295EF10704BEF1030596E
:102770001375F50F2305A420A305A4202285EFF0EF
:102780003FE6A1BF930720046311F90216347E309F
:102790001387F6FF63D8E70085077EB09307A41B75
:1027A0006E304DBF9DDA7AB0D5BF930740046310F9
:1027B000F9028347B42095D313850926EFE02FFF54
:1027C00098408347B720FD17A305F72039B7930733
:1027D0003004E319F9F48347B4200347A420E3FE4F
:1027E000E7EE3E948305A41B13854A26EFE02FFCF9
:1027F00098408347B7208507C1BF13850926EFE0BE
:102800000FFB050980408347B420E348F9FE130518
:102810008AA5EFE0CFF9EFF09FA785471304A41B2B
:102820006315F5002285EFF07FC1EFF0BFD7228658
:10283000AA851385CC27EFE08FF780401305A41BF2
:10284000EF10F04B1375F50F2305A420A305A4206A
:1028500069B59307F0076305F900A1476315F90807
:102860008347B420E38B07E60346A420FD1793F7C4
:10287000F70F7D161376F60F2305C420A305F42069
:1028800063F8C7049385B71B1385A71B1D8EA295FC
:102890002295EFE04FAE9C4013858B2603C7A720FF
:1028A0003E97230D071A83C5B7209385A51BBE95B8
:1028B000EFE0EFEF9C4003C4B7209C4083C7A72004
:1028C000E3CD87E013850926EFE06FEE0504F5B749
:1028D00013050B27EFE0AFED9C4003C7A720BA9785
:1028E000238D071ADDBB35478347A4206305E90024
:1028F0002947631EE90EB9CB035984029147130D92
:10290000A41B63FB2709930DA41613060005EA8593
:102910006E85EF10902E1DC91309A4024A85130974
:10292000090513060005CA85EF10702FE3982DFFE7
:102930001306000581456E85EFD0BFA90346A4208C
:10294000EA856E85EF10B02D95471EB41E347EB01B
:10295000EFF0FF9385476312F5029C4083C747025F
:10296000858B89C713058AA5EFE06FE4884083450E
:10297000A5201305A51BEFF0DF91EFF0BFC2EFE03C
:102980000FE380401306000581451305A41BEFD01B
:102990005FA42315042091B3630109021305F9FF15
:1029A000930700053305F50213060005EA851305B4
:1029B000A5022295EF10702451D9930D000533051F
:1029C000B9031306000581451305A5022295EFD032
:1029D0005FA00A340346A420EA853305B503130536
:1029E000A5022295EF10B0231E348507B9BF130747
:1029F000F0046374F700230504200346B4208347E2
:102A0000A4206370F6089305A61B1305B61BA295B8
:102A10003386C7402295EFE00F968C4083C7B520E0
:102A20003387F500230D271B03C74502058B01CB18
:102A30009387A71BBE9513058CFFEFE04FD79C40F3
:102A400003C4B7209C4083C7A7206346F402984084
:102A50008347A7208346B7208507850693F7F70F9E
:102A6000A305D7202305F7209306F004E3F7F6C665
:102A7000231507209DB113850926EFE04FD30504E8
:102A8000D1B7A297238D271B83474402858BE1D3BF
:102A9000CA8513854A26EFE08FD155BF7C41232894
:102AA0000504232A05049C4381CBEFD29F8F930515
:102AB000850482976FD03F9101458280EFD2DF8CF1
:102AC00036899DCAAA843284B309D600294A1C20BB
:102AD000639B4701BE2C93F7070491C7FC40B545A3
:102AE00026859C478297FC408305040026859C47E9
:102AF00005048297E31D34FD4A856FD03F8CEFD2E9
:102B00005F8A93F705102A8491C71A2D61551377B0
:102B1000071035CF13F7054011C71A2C61551377ED
:102B2000074035C713F705049304000401E7262C7A
:102B300093F40404384893F5F50F2EAC39EBA1C794
:102B400068442981420541813105EFE0EFE5704499
:102B50002A89310529824206418281452320A90024
:102B6000EFD0FFF8232209003E2C2324090023285C
:102B7000240593E707103EAC7C4013060010C145C6
:102B8000DC43228582973E2C0145DD8C26AC6FD03C
:102B90009F83F5DB93E505102EACF5B70948AA87AE
:102BA00063810503EFD2EFFF0D48638205030547FC
:102BB0006399E5041A2D1377F7FD1AAD01456FD01F
:102BC0009F801A2D136707021AAD01458280328754
:102BD00075D6504274454C2D2982A9824206C20600
:102BE0004182C1826304D6001D45F1F91443B4C784
:102BF0005443F4C7E1D5F443BA853E8594428296A6
:102C000075BF7C41DC4382975DBFEFD2EFF736841E
:102C1000B1CA3E2DAA89328993F70710B6849DE385
:102C20007D5AA94A83A749044E85DC4782976309E8
:102C300045012300A900FD14050963035501FDF0BA
:102C4000058C0DA02449368A854AEFE09FF3FE20CB
:102C5000DA202A869444631AF70081EAEFE03FF312
:102C60003304444122856FD06FF598403E97034B63
:102C7000070003A7C9048507C2072983C183420748
:102C8000FEA0418363E4E7002393040063945601AC
:102C900023A404003285EFE09FEF7D1A2300690131
:102CA0000509E3140AFA6DBF582D854763ECE70266
:102CB0003E2D93F707109DC7EFD2AFEE2A84284927
:102CC000EFE08FE33E2C232804041306001093F753
:102CD000F7EF3EAC7C40C5452285DC438297014539
:102CE0006FD06FEE01458280EFD2AFEB3737000037
:102CF0001307C7A918D5373700001307E7AF58D512
:102D000037370000130787CA18D937370000130771
:102D1000A7C058D9373700001307C7AB18DD3737BE
:102D200000001307C7B9420658DD34C14182232A87
:102D300005002320050223220502EFD01F896FD052
:102D40008FE893F5F50F85476391F50AEFD2CFE34E
:102D500020494111AA847D598549FC402685DC47DC
:102D600082972A8A63072505EFE0BFE15A201C40BD
:102D7000BA97238047015E20F8448507C20729835C
:102D8000C18342075EA0418363E4E700231204008D
:102D900076205E20639CD7008507C207C1837EA092
:102DA0002324340163E4E70023130400EFE03FDE53
:102DB0006DB79C5085C3EFE0DFDC5A206E20636E58
:102DC000B700B305B7402EC6EFE07FDC9C50B2459C
:102DD0002685829741016FD06FDEFC44998DA983CF
:102DE000C207C183B385B740F9BF828001CEEFD25D
:102DF0004FDB7841B2878E23184332220297014578
:102E00006FD06FDC7D558280EFD2AFD91387C1CEF2
:102E100078432E86AA8518431385C1CE02976FD0BA
:102E20008FDAEFD20FD81387C1CE78432E86AA85CA
:102E300058431385C1CE02976FD0EFD8EFD26FD62B
:102E40001387C1CE7843AA851385C1CE1847029750
:102E50006FD06FD705C611476392E602EFD26FD4E9
:102E60007C410E2241119C4736C632C482972246CD
:102E7000B2462AA2368541016FD0EFD4814636850D
:102E800082801DC2B28711466390C602EFD26FD115
:102E90007841B2238E235843411136C60297B24679
:102EA000410136856FD02FD2814636858280EFD2A0
:102EB0004FCF9387C1CE4947D8CB37370000130790
:102EC00047E5D8DB37370000130727E898DF3737A7
:102ED00000001307C7DEECC3B0C3AA850D461385F7
:102EE000C1CE23A0070223A2070223A4070223A620
:102EF000070223A80702D8DFEFD02FED01456FD0DE
:102F00008FCC3705002013054569828037150020D6
:102F1000130545698280EFD2CFC8B707002003A709
:102F200007169307803EC1563357F702B7E700E014
:102F30002386D7402387D740856623A0D710916684
:102F400023A0D710B7F700E023A0070023A20700B3
:102F5000014690C78146D4C781461306F7FF90CB40
:102F6000D4CB3D4798C3EFD0AFD7EFF09FF92A8479
:102F7000EFF0DFF9AA852285EFE04F9B375500007F
:102F80001305452FEFD0BFFF6FD0EFC3731101348E
:102F9000EFD07F96B7F700E023A20700EFD04FCE27
:102FA000EFD03F987311013473002030814785467C
:102FB000130700023396F6006306A6008507E39B1D
:102FC000E7FEFD573E858280EFD2AFBD85451305F4
:102FD0000002EF0090736FD00FBFEFD28FBC85451A
:102FE0002145EF0090726FD00FBEEFD28FBB8545A9
:102FF0001145EF0090716FD00FBDEFD28FBA8545AC
:103000004145EF0090706FD00FBCEFD28FB985456E
:1030100013050004EF00706F6FD0EFBAEFD26FB8F6
:1030200095653765000001469385C52F1305459EBC
:10303000EFF0FFE76FD02FB99307400663ECA700CE
:10304000931745001565130545393E951841FD5701
:103050006313F70001458280EFD2AFB4411113F53D
:10306000F50F32C6EFF05FFD11C54E25324608451B
:10307000EF00104A41016FD00FB5EFD28FB213F5B8
:10308000F50FEFF07FFBAA87014589C7CE27884758
:10309000EF0070476FD02FB3EFD2AFB0011113F52F
:1030A000F50F3284EFF05FF905C55C412AC68297BF
:1030B00032455C45FC82C1473ECE8D473ECC09C4BB
:1030C0001547631AE40002CE08454C08EF00B037FC
:1030D00005616FD04FAF05476315E40091473ECEC1
:1030E000E5B76315F40093078002D5BF89476315E0
:1030F000F40093078004E5B791476314F400D147C7
:10310000F9BF99476314F400F147D1BF9D47E31D10
:10311000F4FAE147E9B7EFD22FA713F5F50FAE8424
:10312000B289368A3A89EFF03FF1994731CD484567
:10313000EFF0DFE73D472A8499476367A704EFE094
:103140005FA4B146B306D402B7070020138707086F
:103150002A8693870708369783160700639F960091
:103160004C43639C45012E23639935011847631630
:103170002701EFE0DFA1814701A87D576389E600C1
:103180003285EFE0DFA09D473E856FD02FA331450C
:103190003305A4023E9506A12322450123113501E2
:1031A000232425013285F1B7EFD2AF9F13F5F50F38
:1031B000EFF09FE819471DC94845EFF03FDFBD47D5
:1031C0002A84194763E4A702EFE0BF9BB1473304A9
:1031D000F402B7070020938707087D57A2978396CC
:1031E00007006398E600EFE09F9A01473A856FD0A9
:1031F0008F9D41677D1798C323A2070023A4070072
:10320000DDB7EFD26F98011113F5F50F328AEFF0A9
:10321000BFE2994721C185442A8463159A10484525
:10322000EFF0DFD83D47AA8499476365A702EFE036
:103230005F95B14AB3875403370900201309090881
:10324000AA893E9903170900FD576319F700EFE0BB
:103250001F9499473E8505616FD04F965C408297D9
:1032600085450545EF00704A5C440D473AC47C82B1
:103270003EC88357290002CA52CE638C4709C1C792
:103280000947638DE70808444C00EF00D01B184441
:10329000B7170140938607C005456302D702094569
:1032A000630FF700938707400D45630AF700B727C0
:1032B00001409387078001456313F700114593F59B
:1032C000F40FEF0090250808EF00D00E9567938764
:1032D00047318E04BE94D04037E700E093060005E6
:1032E000B307C7002380D74093575600938707043E
:1032F00085468A07B396C600BA9794C34E85EFE019
:103300001F89814781BF930780023EC6A1473ECCFB
:103310009DBF930780043EC656CCB5B791473EC6C5
:10332000C147F5B79947E3170AF24845EFF01FC8C0
:103330003D479947E360A7F29317350015651305DC
:1033400045313E9558419357570093870706B394EC
:10335000E4008A0737E700E0BA9784C35DB7EFD28D
:103360004F84EFF0BFC4B1473305F502B707002023
:10337000938707083E955C4199C3084582976FD0B3
:103380008F8473110134EFD00FD70545EF0030095A
:1033900019C50545EFF0BFFC0545EF00300AEFD039
:1033A0004FD8731101347300203073110134EFD002
:1033B0008FD40945EF00B00619C50945EFF03FFA73
:1033C0000945EF00B007EFD0CFD57311013473007A
:1033D000203073110134EFD00FD21145EF003004CB
:1033E00019C51145EFF0BFF71145EF003005EFD0DB
:1033F0004FD3731101347300203073110134EFD0B7
:103400008FCF2145EF00B00119C52145EFF03FF501
:103410002145EF00B002EFD0CFD07311013473001B
:10342000203073110134EFD00FCD4145EF00207FE4
:1034300019C54145EFF0BFF24145EF003000EFD034
:103440004FCE731101347300203073110134EFD06B
:103450008FCA13050002EF00807C1DCD130500020A
:10346000EFF0FFEF13050004EFF07FEF1305000806
:10347000EFF0FFEE13050010EFF07FEE13050020D4
:10348000EFF0FFED1305003EEF00407BEFD06FC97A
:10349000731101347300203013050004EF0020780D
:1034A00055FD13050008EF0080774DF91305001056
:1034B000EF00E07645F513050020EF00407659FD5A
:1034C000F1B773110134EFD00FC313050040EF00C3
:1034D000007529C113050040EFF07FE8056513056D
:1034E0000580EFF0DFE70565EFF07FE70965EFF0B6
:1034F0001FE71165EFF0BFE62165EFF05FE641657C
:10350000130505C0EF008073EFD0AFC17311013414
:1035100073002030056513050580EF0040705DF9EC
:103520000565EF00C06F5DF50965EF00406F5DF167
:103530001165EF00C06E59FD2165EF00406E59F92D
:10354000E1B701458280EFC2DFE59C412041A14601
:1035500041111CC0B1473EA4DC412316040013F7FF
:10356000F7006301D702A546631ED70005675AA07E
:1035700013D747000D8B01C785466308D700231377
:10358000040031A023120400E5B709677AA09983EB
:103590008D8B05476389E70081C709476387E70685
:1035A0002314040021A0930700601EA41848B74705
:1035B0000140938707806316F7041165854511055F
:1035C000EF00B01493070020B71401407C820D492E
:1035D000E1474C00138504803EC64AC4AD259307DD
:1035E00000407C824C009147138504803EC64AC44B
:1035F000992D0848A285EF00101508488545EF0071
:10360000901D014541016FC01FDC9307004071BF51
:10361000EFC29FD7B71400201384C46E93075003E2
:103620005CC837190020B7470140130649699387E2
:10363000078074461CC899679387879E7CC2B7072A
:1036400000C0F58FC166A106716713070720D58FEB
:103650001165411138C67CC68545B7070C001105B8
:1036600018C01CC42322040023160400EF00F00934
:10367000B7190140930700207C820D4AE1474C00B6
:103680001385098052C43EC67D2B930700407C827F
:103690004C009147138509803EC652C46D230848EB
:1036A0009385C46EEF00300A08488545EF00B012DC
:1036B000B75500009386C46E130630109385452FCE
:1036C00013054969EFF04FE2014541016FC01FCF7B
:1036D000EFC23FCD2041930500020848EF0070156E
:1036E00019C51C48CA231375F50F6FC0DFCD7D5572
:1036F000EDBFEFC21FCB24412E8488489305000400
:10370000EF0030137DD99C4842044180C2A3054597
:103710006FC07FCBEFC2FFC8C1473841638BF50252
:10372000C5476395F502544B054693D756009387DA
:1037300007063316D6008A07B7E600E0B69790C3AF
:103740000146084B93055052EF00500A01456FC0E7
:103750009FC7544B054693D75600938707043316EB
:10376000D6008A07B7E600E0B69790C30546D1BFFA
:10377000411122C626C473110134B7140020EFD0C2
:103780008F9793874469A043930550520848EF00F0
:10379000B00B19C9854513854469EFF08FDA0848E5
:1037A00093055052EF00100EEFD0AF977311013414
:1037B0003244A24441017300203073110134EFD030
:1037C0008F9337650000130585A0EFD04FFEEFD033
:1037D0004F95731101347300203073110134EFD011
:1037E0008F91376500001305C59FEFD04FFCEFD0D8
:1037F0004F937311013473002030EFC29FBA3765C5
:103800000000130585A1EFD08FFA992AB707002091
:1038100083A50716376500001305C5A2EFD02FF961
:103820006926AA85376500001305C5A3EFD02FF8D8
:10383000376500001305C5A4EFD06FF731280145A7
:103840006FC07FB8EFC2FFB5EF001005EF00D005E5
:10385000EF00301A6FC03FB7EFC2BFB4EFF09FFE6A
:10386000C5246FC05FB6B71702409843B706FFF094
:1038700041111367170098C3D84337060200758FAC
:10388000D8C39843B706F7FEFD16758F98C39843C3
:10389000B706FCFFFD16758F98C3D843B70601FF26
:1038A000FD16758FD8C39843B70600ECFD16758FCB
:1038B00098C33707FF0098C723A6070202C402C6B1
:1038C0009843C166558F98C3B716024005679C425E
:1038D000F18F3EC6A24785073EC4B24781E7A247A3
:1038E000E397E7FEB71702409C431397E70063573F
:1038F000070685473EC632478547631FF704B7175B
:103900000240D843B706C1FFFD16D8C3D843D8C379
:10391000D84313670740D8C3D843758FD8C3D8435B
:10392000B7062900558FD8C39843B7060001558FB5
:1039300098C3984393166700E3DD06FED843B71695
:103940000240719BD8C3D84313672700D8C32147CF
:10395000DC42B18BE39EE7FE4101828002C661BF7B
:10396000B7160240D842B70700201146318B938723
:1039700007166305C70021466308C70237177A0098
:103980001307072098C337170240584311839376D3
:10399000F7003707002013070714369714239843BE
:1039A0003357D70098C38280D842D44241664983B6
:1039B0003D8BF18E1306270015CF3D47630FE602BE
:1039C0004147630FE602454781456313E6004146E0
:1039D000A1E23747024003270780418B0DC7371705
:1039E0007A00130707203306C70290C3C9DD984346
:1039F000058349BF81454946E1BF85453546C9BF75
:103A000081453D46F1B737173D0013070790E1BFE9
:103A10003715024058559316F700585563DF0604D2
:103A200011833D8B9306170037177A001307072081
:103A30003357D70298C35455A182BD8A8DE295466B
:103A40003307D702058398C337170240585794436A
:103A50003D8B050733D7E60298C3984369B7054500
:103A60006394A600E546E9BF3D456396A600D146AE
:103A70003387E602C9BF8906E5BF3D8B9306170071
:103A800037177A00130707203357D702F1B701A081
:103A90007390123497D1FF1F9381C1EC17C100209E
:103AA00013014156172500001305451497C5FF1F44
:103AB000938545551386818063FAC50083220500EE
:103AC00023A0550011059105E3EAC5FE1385818009
:103AD00097E5FF1F938545D56377B5002320050043
:103AE0001105E36DB5FEFD42739002BCFD4273907B
:103AF0004280B7820000938202807390023097C2A6
:103B0000FFFF9382625093E2320073905230EFF0E5
:103B10009FD597D2FFFF938262A6739012347300F1
:103B20002030EFC21F88B75400400564938404809E
:103B3000130484BB26851D282285EFD09FD9DDBFC5
:103B4000EFC23F86B745000037650000D1472947DF
:103B5000930600200146938525B21305C5A5EFD035
:103B60003FC519C1EFD09FDC6FC0FF85EFC27F83D7
:103B7000B7150020156793874570130737C59AA3BB
:103B80007D57BAA37D57D8C37577130707EA375512
:103B900000409AA72D465947938545701305058027
:103BA000B8A7EF00E0776FC01F82B7F7FF1F03A52C
:103BB000477082805841032805004C453706014074
:103BC000930706403E979346F8FFB1C5832506400C
:103BD000F58D2320B640D043F18ED4C31443B3E611
:103BE000060114C3184190479346F7FF758E90C79E
:103BF000D047F18ED4C7144541466399C600944717
:103C0000D98E94C7D447558FD8C78280B69794432E
:103C1000558F98C382801C43F58F1CC38280B707E1
:103C200001401387074083A70740584B698F09C796
:103C30007D8D3335A000828001458280B707014029
:103C400023AAA74082809C4513F7070113F8F700C9
:103C500001C7D8413368E8008E2113F7F50F39C347
:103C600018418146854E3D4F930F80029302800498
:103C7000214E3396DE00B3F8C50063111603939806
:103C8000260033131F011343F3FF3377E300B31808
:103C9000180133E7E800639FF70550C98506E39AEA
:103CA000C6FD18C11307F00F6375B70454412146D0
:103CB000854E3D4F930F800293028004414EB3988E
:103CC000CE0033F715016392E8021317260001179F
:103CD0003313EF001343F3FFB376D3003317E80039
:103CE000D98E639DF701232A15010506E319C6FD48
:103CF00054C18280E39457FA10C94DB7E39757FE39
:103D000023281501DDB708456D8D3335A00082806D
:103D100019C20CC982804CC9828013F7C50F93F772
:103D20003500B7050140BA9594458A073D473317DA
:103D3000F7001347F7FF758F98C598453315F500C1
:103D4000598D88C5828003A7018B89471021631193
:103D5000F70214318D4763EDD7003C219A0637E70F
:103D600000E09607D58F93F7F70F32972300F740BF
:103D700054410547935756003317C70089CA9387A4
:103D800007048A07B7E600E0B69798C38280938756
:103D90000706C5BF371702405C439146B18B638568
:103DA000D700A1466382D706B7177A00938707200A
:103DB0001CC1371602405C42370700201307071565
:103DC0009183BD8BBA9794231C41B3D7D7005CC1B4
:103DD0005442A1829D8ABA969422B3D6D70014C5C4
:103DE0005442AD829D8A36971823B3D7E7005CC54D
:103DF00058423983937637001387418036971823CA
:103E0000B3D7E7021CC982805C435843C166C983AB
:103E1000758FB7F6FF1F83A6C670BD8B89071396F3
:103E2000160163480600C54601466392D702C9479A
:103E300039A88946638FD702BD46638ED702C14633
:103E4000638ED702C54601466393D700C1471DEF75
:103E50003747024003270780418B05C737177A0091
:103E600013070720B307F7021CC121D61C41858325
:103E700081B701466DBF0546B547D1BF0146BD4775
:103E8000F9B737173D0013070790E9BFB715024090
:103E9000D8559316F700D85563DF060411833D8B80
:103EA0009306170037177A00130707203357D702F6
:103EB00018C1D455A182BD8A8DE295463307D70239
:103EC000058318C137170240585714413D8B050729
:103ED00033D7E60218C1184171B785456394B6001F
:103EE000E546E9BFBD456396B600D1463387E60295
:103EF000C9BF8906E5BF3D8B9306170037177A00C7
:103F0000130707203357D702F1B799C53717024077
:103F10001C4F5D8D08CF8280B7170240984F134524
:103F2000F5FF798D88CF828099C5371702405C4FA5
:103F30005D8D48CF8280B7170240D84F1345F5FFFB
:103F4000798DC8CF8280EFC2CFC51629F577FD17CE
:103F5000F58FF621DA257971D58F1EA95625FD77C3
:103F60009387379FF58FD6212A842EC6D58F962525
:103F7000D58FB625D58F5EA55E29C207C18393F77D
:103F8000F7CFD98F5EA96808EFF0DFE0B7470140AF
:103F900093870780B245631EF402A2576547B38733
:103FA000E7029841930640060A07B3D7E70233D7E2
:103FB000D702B3F7D7021207920793872703B3D725
:103FC000D702BD8BD98FC207C1831EA445616FC0C4
:103FD0008FBF9257E1B791C55E250967D98F5EA55E
:103FE00082805A25F977FD17F98FD5BF13F7F50FA2
:103FF00085471583B395B7006319F7009307C5008C
:10400000984301CED98D8CC38280894693074501A0
:10401000E318D7FE93070501E5B793C5F5FFF98DC2
:10402000DDB793F5F51F4EA182804A211375F51F68
:1040300082800A216D8D3335A000828093C5F5FF03
:10404000C205C1810EA1828013F7F50F8546158345
:10405000B397B6006311D7025A25F98F1A2101458B
:104060004207418381CB0545A181B315B5006D8F12
:104070003335E000828089466314D7001A29F1BFE6
:104080005A29E1BFA1818547B397B70093C7F7FFCE
:10409000C207C1831EA18280EFC2AFB0814509452E
:1040A000EFE09FD66FC02FB2EFC2AFAF8545094595
:1040B000EFE03FD76FC02FB1411122C63754004007
:1040C000930550521305048026C4EFF0FFF705C195
:1040D00013050480EFF07FF51387418B1423B71786
:1040E000002093874772B697850688A314A3B75418
:1040F00000409305404213850480EFF0FFF405C9AA
:104100001384418B1020B7150020938545721385C9
:10411000048039240C2037650000130505A6EFC084
:104120001FE91385048023000400EFF01FF03754CB
:104130000040A14513050480EFF0BFEF8547631BE6
:10414000F50013050480A145EFF05FEF130504802F
:10415000EFF0BFED3244A244410173002030EFC2C2
:104160004FA481451305A002EFE0BFCB6FC0AFA500
:10417000EFC22FA381451305B002EFE09FCA6FC0C5
:104180008FA4EFC20FA281451305C002EFE07FC9E3
:104190006FC06FA3EFC2EFA081451305D002EFE01F
:1041A0005FC86FC04FA2EFC2CF9F81451305E002E9
:1041B000EFE03FC76FC02FA1EFC2AF9EEFF03FFA15
:1041C000EFF01FFBEFF0FFFBEFF0DFFCEFF0BFFDC8
:1041D000814513058003EFE0DFC48145130590039B
:1041E000EFE03FC481451305A003EFE09FC36FC01C
:1041F0008F9DEFC20F9B797181451305A002EFE0FF
:10420000BFC081451305B002EFE01FC08145130513
:10421000C002EFE07FBF81451305D002EFE0DFBEB3
:1042200081451305E002EFE03FBE814513057003B1
:10423000EFE09FBD814513057003EFE09FBE814510
:1042400013058003EFE05FBC814513059003EFE0A9
:10425000BFBB81451305A003EFE01FBBEFF0DFF507
:1042600085452145EFF07FCA854537050400EFF00D
:10427000BFCB93070040FC82371401408D473ECCF2
:104280004C08E147130504C03ECEEFF0DF9B856785
:1042900093870780FC824C089147130504C03ECEEB
:1042A000EFF07F9AF16737540040938707200C1096
:1042B0003ED013050480B7070C003ED402D223166B
:1042C0000102EFF05FC8930770137C8685475C8717
:1042D000680085473EC8EFF01FA713050480054618
:1042E00093055052EFF09FD00546130504809305C7
:1042F0004042EFF0BFCF854513050480EFF0BFCDFE
:1043000045616FC04F8CEFC2CF892A84EFF07FD117
:10431000930500082285EFF0DFD17DD96FC0AF8A09
:10432000EFC28F86B7570040938707802A84AE89F3
:1043300032896316F504854513057003EFE07FAEFF
:10434000CA84B307994093F7F70FCE978C23228541
:10435000FD14EFF05FFBF5F4930500042285EFF008
:104360005FCD7DD9B7570040938707806318F40469
:10437000814513057003EFE0DFAA6FC02F84B727D4
:104380000040138707806315E500854511457DB71B
:10439000138707C06315E5008545154545B73747C1
:1043A0000040130707406315E5008545614579B76F
:1043B000E315F5FC85451305300249B7B7270040E2
:1043C000138707806315E400814511456DB7138796
:1043D00007C06315E4008145154571BF37470040AC
:1043E000130707406315E4008145614569B7E3168B
:1043F000F4F8814513053002BDBF01476314E600A0
:1044000001458280B307E5000507B386E5009C23DC
:1044100083C6F6FFE384D7FE3385D7408280B3C7D7
:10442000A5008D8B3307C50081E78D4763EDC7007D
:10443000AA87637EE508942185078505A38FD7FEAB
:10444000E3EBE7FE828093763500AA8789CA942140
:1044500085078505A38FD7FE93F63700C5BF9376F2
:10446000C7FF138606FE63F0C70683A3050083A279
:10447000450083AF850003AFC50083AE050103AEE1
:10448000450103A3850183A8C5019385450223A0A7
:10449000770003A8C5FF23A2570023A4F70123A692
:1044A000E70123A8D70123AAC70123AC670023AEE5
:1044B00017019387470223AE07FF75B79041910715
:1044C000910523AEC7FEE3EBD7FEE3E6E7F6828075
:1044D000AA8798239386170009EB850503C7F5FF84
:1044E0008507A38FE7FE75FB8280B687DDB7AA87B5
:1044F000982185078505A38FE7FE7DFB8280AA872B
:10450000850703C7F7FF6DFF3385A7407D158280C0
:1045100015C27D160147B307E500B386E5009C236D
:1045200094226396D7006304C7000507EDF733852F
:10453000D740828001458280005000001450000066
:10454000245000003850000044500000505000003B
:104550005450000064500000745000007C50000073
:1045600090500000A0500000A8500000B45000007F
:10457000C0500000D4500000DC500000EC5000009F
:10458000FC500000145100006D61696E00000000D5
:10459000546F20696E697469616C697A652064651D
:1045A000766963653A2573206661696C65642E20BF
:1045B000546865206572726F7220636F646520694C
:1045C000732025640A0000007469646C65000000B3
:1045D00000000100020001000300010002000100D0
:1045E00004000100020001000300010002000100BC
:1045F00005000100020001000300010002000100AB
:10460000040001000200010003000100020001009B
:104610000600010002000100030001000200010089
:10462000040001000200010003000100020001007B
:10463000050001000200010003000100020001006A
:10464000040001000200010003000100020001005B
:104650000700010002000100030001000200010048
:10466000040001000200010003000100020001003B
:10467000050001000200010003000100020001002A
:10468000040001000200010003000100020001001B
:104690000600010002000100030001000200010009
:1046A00004000100020001000300010002000100FB
:1046B00005000100020001000300010002000100EA
:1046C00004000100020001000300010002000100DB
:1046D0003031323334353637383941424344454638
:1046E000000000000A205C207C202F0A000000004F
:1046F0002D205254202D20202020205468726561E6
:1047000064204F7065726174696E672053797374A9
:10471000656D0A004A756E20313320323032340024
:10472000202F207C205C202020202025642E256442
:104730002E2564206275696C642025730A000000D0
:104740002032303036202D203230313920436F7006
:104750007972696768742062792072742D74687246
:10476000656164207465616D0A000000284E554C37
:104770004C290000303132333435363738396162F4
:104780006364656600000000746F74616C206D6581
:104790006D6F72793A2025640A00000075736564B4
:1047A000206D656D6F7279203A2025640A00000043
:1047B0006D6178696D756D20616C6C6F6361746596
:1047C00064206D656D6F72793A2025640A000000DF
:1047D0006C697374206D656D6F7279207573616794
:1047E0006520696E666F726D6174696F6E0000009E
:1047F0006C6973745F6D656D00000000746F2066F6
:104800007265652061206261642064617461206268
:104810006C6F636B3A0A00006D656D3A2030782545
:104820003038782C207573656420666C61673A2097
:1048300025642C206D6167696320636F64653A208D
:104840003078253034780A00686561700000000017
:104850006D656D20696E69742C206572726F7220AF
:10486000626567696E206164647265737320307875
:1048700025782C20616E6420656E6420616464720A
:1048800065737320307825780A0000001B5B324A7C
:104890001B5B48002D2D46756E6374696F6E204C4E
:1048A0006973743A0A0000005F5F0000252D3136FD
:1048B00073202D2D2025730A0000000064657669A1
:1048C00063650000252D2A2E732020202020202023
:1048D0002020747970652020202020202020207244
:1048E000656620636F756E740A000000202D2D2D03
:1048F0002D2D2D2D2D2D2D2D2D2D2D2D2D2D2D2DE8
:104900002D202D2D2D2D2D2D2D2D2D2D0A0000008E
:10491000252D2A2E2A7320252D32307320252D385F
:10492000640A00006576656E74000000252D2A2E4D
:104930007320202020202073657420202020737590
:104940007370656E64207468726561640A000000AB
:1049500020202D2D2D2D2D2D2D2D2D2D202D2D2DAE
:104960002D2D2D2D2D2D2D2D2D2D2D0A000000004E
:10497000252D2A2E2A7320203078253038782025BE
:104980003033643A00000000252D2A2E2A7320209F
:1049900030782530387820300A0000006D61696C6D
:1049A000626F7800252D2A2E7320656E747279202F
:1049B00073697A652073757370656E6420746872AC
:1049C0006561640A00000000202D2D2D2D20202D72
:1049D0002D2D2D202D2D2D2D2D2D2D2D2D2D2D2D14
:1049E0002D2D0A00252D2A2E2A73202530346420EF
:1049F00020253034642025643A000000252D2A2E1D
:104A00002A73202530346420202530346420256426
:104A10000A0000006D736771756575650000000020
:104A2000252D2A2E7320656E74727920737573702C
:104A3000656E64207468726561640A00202D2D2DF6
:104A40002D20202D2D2D2D2D2D2D2D2D2D2D2D2DB0
:104A50002D0A0000252D2A2E2A73202530346420AB
:104A60002025643A00000000252D2A2E2A732025D7
:104A7000303464202025640A000000006D757465E0
:104A800078000000252D2A2E732020206F776E6578
:104A9000722020686F6C642073757370656E64207B
:104AA0007468726561640A00202D2D2D2D2D2D2D29
:104AB0002D202D2D2D2D202D2D2D2D2D2D2D2D2D40
:104AC0002D2D2D2D2D0A0000252D2A2E2A7320256F
:104AD0002D382E2A7320253034642025640A0000E6
:104AE00073656D6170686F7265000000252D2A2E58
:104AF00073207620202073757370656E642074684F
:104B0000726561640A000000202D2D2D202D2D2DB1
:104B10002D2D2D2D2D2D2D2D2D2D2D0A000000009C
:104B2000252D2A2E2A7320253033642025643A004F
:104B3000252D2A2E2A7320253033642025640A006F
:104B40007468726561640000252D2A2E73207072CE
:104B500069202073746174757320202020202073D5
:104B6000702020202020737461636B2073697A6544
:104B7000206D61782075736564206C65667420749F
:104B800069636B20206572726F720A00202D2D2DD3
:104B900020202D2D2D2D2D2D2D202D2D2D2D2D2D6C
:104BA0002D2D2D2D202D2D2D2D2D2D2D2D2D2D204F
:104BB000202D2D2D2D2D2D20202D2D2D2D2D2D2D4C
:104BC0002D2D2D202D2D2D0A00000000252D2A2E03
:104BD0002A732025336420002072656164792020C7
:104BE000000000002073757370656E6400000000A3
:104BF00020696E69742020200000000020636C6F23
:104C0000736520200000000020307825303878209F
:104C10003078253038782020202025303264252532
:104C200020202030782530387820253033640A0061
:104C300074696D6572000000252D2A2E7320207086
:104C40006572696F64696320202074696D656F7592
:104C50007420202020202020666C61670A0000005C
:104C6000202D2D2D2D2D2D2D2D2D2D202D2D2D2D8E
:104C70002D2D2D2D2D2D202D2D2D2D2D2D2D2D2D71
:104C80002D2D0A00252D2A2E2A7320307825303824
:104C9000782030782530387820000000616374690E
:104CA00076617465640A00006465616374697661A5
:104CB0007465640A0000000063757272656E74208A
:104CC0007469636B3A3078253038780A0000000048
:104CD0006C69737420616C6C2073796D626F6C20E9
:104CE000696E2073797374656D0000006C6973746C
:104CF000000000006C697374206465766963652048
:104D0000696E2073797374656D0000005F5F636D79
:104D1000645F6C6973745F64657669636500000045
:104D20006C6973742064657669636520696E2073AD
:104D3000797374656D0000006C6973745F646576E7
:104D4000696365006C6973742074696D65722069AC
:104D50006E2073797374656D000000005F5F636D92
:104D6000645F6C6973745F74696D65720000000044
:104D70006C6973742074696D657220696E20737933
:104D80007374656D000000006C6973745F74696D05
:104D9000657200006C697374206D6573736167657B
:104DA00020717565756520696E2073797374656D02
:104DB000000000005F5F636D645F6C6973745F6D1A
:104DC00073677175657565006C697374206D6573C3
:104DD0007361676520717565756520696E207379EB
:104DE0007374656D000000006C6973745F6D7367A8
:104DF00071756575650000006C697374206D61697B
:104E00006C20626F7820696E2073797374656D0011
:104E10005F5F636D645F6C6973745F6D61696C6221
:104E20006F7800006C697374206D61696C20626F2B
:104E30007820696E2073797374656D006C69737482
:104E40005F6D61696C626F78000000006C6973745B
:104E5000206D7574657820696E2073797374656D43
:104E6000000000005F5F636D645F6C6973745F6D69
:104E700075746578000000006C697374206D75743A
:104E8000657820696E2073797374656D0000000089
:104E90006C6973745F6D7574657800006C69737408
:104EA000206576656E7420696E2073797374656D04
:104EB000000000005F5F636D645F6C6973745F6521
:104EC00076656E74000000006C6973742065766509
:104ED0006E7420696E2073797374656D0000000034
:104EE0006C6973745F6576656E7400006C697374C9
:104EF0002073656D6170686F726520696E207379CB
:104F00007374656D000000005F5F636D645F6C69C2
:104F100073745F73656D00006C6973742073656DE5
:104F20006170686F6E6520696E2073797374656D4A
:104F3000000000006C6973745F73656D0000000011
:104F40006C69737420746872656164005F5F636D7F
:104F5000645F6C6973745F746872656164000000FB
:104F60006C69737420746872656164006C69737431
:104F70005F74687265616400746865207465726D41
:104F8000696E616C2073637265656E005F5F636D4F
:104F9000645F636C65617200746865207465726D2E
:104FA000696E616C2073637265656E00636C656128
:104FB000720000007265626F6F7420746865206211
:104FC0006F617264000000005F5F636D645F726513
:104FD000626F6F74000000007265626F6F742074FE
:104FE000686520626F617264000000007265626F24
:104FF0006F7400002D000000257300002F000000DA
:1050000043686172616374657220446576696365A3
:1050100000000000426C6F636B2044657669636535
:10502000000000004E6574776F726B20496E7465E6
:1050300072666163650000004D54442044657669E2
:105040006365000043414E20446576696365000056
:1050500052544300536F756E6420446576696365EE
:1050600000000000477261706869632044657669DA
:105070006365000049324320427573005553422056
:10508000536C6176652044657669636500000000B5
:1050900055534220486F737420427573000000001E
:1050A0005350492042757300535049204465766936
:1050B000636500005344494F2042757300000000AF
:1050C000504D2050736575646F2044657669636543
:1050D000000000005069706500000000506F72749D
:1050E000616C2044657669636500000054696D65F4
:1050F0007220446576696365000000004D69736342
:10510000656C6C616E656F75732044657669636567
:1051100000000000556E6B6E6F776E00546F6F204D
:105120006D616E7920617267732021205765206F51
:105130006E6C79205573653A0A00000025732000D3
:1051400025733A20636F6D6D616E64206E6F7420FD
:10515000666F756E642E0A0052542D546872656134
:1051600064207368656C6C20636F6D6D616E647331
:105170003A0A00005F5F636D645F0000252D3136E1
:1051800073202D2025730A0052542D5468726561D6
:1051900064207368656C6C2068656C7000000000AA
:1051A0005F5F636D645F68656C70000053686F7764
:1051B00020746865206D656D6F7279207573616705
:1051C0006520696E207468652073797374656D005D
:1051D0005F5F636D645F6672656500004C69737440
:1051E000207468726561647320696E20746865203C
:1051F00073797374656D00005F5F636D645F7073D6
:10520000000000006D7368200000000066696E7386
:10521000682000003E00000066696E73683A2063F3
:10522000616E206E6F742066696E642064657669B5
:1052300063653A2025730A006E6F206D656D6F728D
:105240007920666F72207368656C6C0A000000003C
:10525000747368656C6C00007368727800000000FD
:1052600008000000256300000825732020080000C6
:10527000082008001B5B324B0D00000025732573CE
:10528000000000007265616420737461747573209E
:1052900066726F6D206861726477617265207069F3
:1052A0006E00000070696E52656164007772697407
:1052B000652076616C756520746F20686172647713
:1052C0006172652070696E0070696E5772697465ED
:1052D0000000000073657420686172647761726514
:1052E0002070696E206D6F646500000070696E4DFE
:1052F0006F646500756172743100000098300000C1
:10530000583000007A30000016310000A83100004B
:105310000232000001000000160000000200000040
:105320001700000004000000180000000800000042
:1053300019000000100000001A000000200000000A
:10534000270000004000000027000000800000004F
:1053500027000000000100002700000000020000FC
:1053600027000000000400003800000000080000D2
:10537000380000000010000038000000002000008D
:1053800038000000004000003800000000800000ED
:1053900038000000FFFFFFFF0000000000000000D9
:1053A00000000000010000000A3000000018014069
:1053B00004000000020000000A3000000018014054
:1053C00008000000030000000A300000001801403F
:1053D00010000000040000000A3000000018014026
:1053E00020000000050000000A3000000018014005
:1053F00040000000FFFFFFFF000000000000000071
:105400000000000007000000FA2F0000001001401B
:105410000020000008000000FA2F000000100140EA
:105420000040000009000000FA2F000000100140B9
:1054300000800000FFFFFFFF0000000000000000F0
:1054400000000000FFFFFFFF000000000000000060
:1054500000000000FFFFFFFF000000000000000050
:1054600000000000FFFFFFFF000000000000000040
:1054700000000000FFFFFFFF000000000000000030
:10548000000000000F000000FA2F00000010014093
:105490000100000010000000FA2F00000010014081
:1054A0000200000011000000FA2F0000001001406F
:1054B0000400000012000000FA2F0000001001405C
:1054C00008000000FFFFFFFF0000000000000000D8
:1054D00000000000FFFFFFFF0000000000000000D0
:1054E00000000000FFFFFFFF0000000000000000C0
:1054F00000000000FFFFFFFF0000000000000000B0
:105500000000000017000000EA2F00000008014022
:105510000100000018000000EA2F00000008014010
:105520000200000019000000EA2F000000080140FE
:10553000040000001A000000EA2F000000080140EB
:1055400008000000FFFFFFFF000000000000000057
:1055500000000000FFFFFFFF00000000000000004F
:10556000000000001D000000EA2F000000080140BC
:10557000100000001E000000EA2F0000000801409B
:10558000200000001F000000EA2F0000000801407A
:105590004000000020000000EA2F00000008014049
:1055A0008000000021000000FA2F000000100140E0
:1055B0001000000022000000FA2F0000001001403F
:1055C0002000000023000000DA2F0000000C014042
:1055D0000100000024000000DA2F0000000C014050
:1055E0000200000025000000DA2F0000000C01403E
:1055F00004000000260000000A30000000180140EE
:1056000080000000270000000A3000000018014060
:1056100000010000280000000A30000000180140CE
:1056200000020000290000000A30000000180140BC
:10563000000400002A0000000A30000000180140A9
:10564000000800002B0000000A3000000018014094
:10565000001000002C0000000A300000001801407B
:10566000002000002D0000000A300000001801405A
:10567000004000002E0000000A3000000018014029
:10568000008000002F000000DA2F0000000C014015
:105690000004000030000000DA2F0000000C014080
:1056A00000080000FFFFFFFF0000000000000000F6
:1056B00000000000FFFFFFFF0000000000000000EE
:1056C0000000000033000000DA2F0000000C014051
:1056D0000010000034000000DA2F0000000C014030
:1056E0000020000035000000DA2F0000000C01400F
:1056F0000040000036000000DA2F0000000C0140DE
:105700000080000037000000C82F00000014014096
:105710000001000038000000C82F00000014014004
:105720000002000039000000C82F000000140140F2
:10573000000400003A000000C82F000000140140DF
:10574000000800003B000000C82F000000140140CA
:10575000001000003C000000C82F000000140140B1
:10576000002000003D000000C82F00000014014090
:10577000004000003E000000C82F0000001401405F
:10578000008000003F000000FA2F000000100140E0
:105790004000000040000000FA2F0000001001400F
:1057A0008000000041000000FA2F000000100140BE
:1057B0000001000042000000FA2F0000001001402C
:1057C0000002000043000000EA2F00000008014032
:1057D0000001000044000000EA2F00000008014022
:1057E0000002000045000000EA2F00000008014010
:1057F0000004000046000000EA2F000000080140FD
:105800000008000047000000EA2F000000080140E7
:105810000010000048000000EA2F000000080140CE
:1058200000200000FFFFFFFF00000000000000005C
:1058300000000000FFFFFFFF00000000000000006C
:1058400000000000FFFFFFFF00000000000000005C
:10585000000000004C000000EA2F0000000801409A
:10586000004000004D000000EA2F00000008014049
:10587000008000004E000000FA2F000000100140E0
:10588000000400004F000000FA2F0000001001404B
:105890000008000050000000FA2F00000010014036
:1058A0000010000051000000C82F0000001401404B
:1058B0000100000052000000C82F00000014014049
:1058C0000200000053000000C82F00000014014037
:1058D0000400000054000000C82F00000014014024
:1058E0000800000055000000C82F0000001401400F
:1058F0001000000056000000C82F000000140140F6
:105900002000000057000000C82F000000140140D4
:105910004000000058000000C82F000000140140A3
:105920008000000059000000DA2F0000000C014048
:10593000080000005A000000DA2F0000000C0140AF
:10594000100000005B000000DA2F0000000C014096
:10595000200000005C000000DA2F0000000C014075
:10596000400000005D000000DA2F0000000C014044
:1059700080000000FFFFFFFF0000000000000000AB
:10598000000000005F000000DA2F0000000C014062
:105990000001000060000000DA2F0000000C014050
:1059A00000020000610000000A3000000018014001
:1059B00001000000620000000A30000000180140F1
:1059C00002000000FFFFFFFF0000000000000000D9
:1059D00000000000FFFFFFFF0000000000000000CB
:1059E0000000000070696E004635000014370000AA
:1059F000F2360000D03600004235000020686172A7
:105A00006466756C740D0A00204E4D492048616E25
:105A1000646C65720D0A00000D0A204D43553A2052
:105A200043483332563330330D0A00002053797324
:105A3000436C6B3A202564487A0D0A00204368695C
:105A40007049443A20253038780D0A00207777775E
:105A50002E7763682E636E0D0A0000006C6564008B
:105A600055534152545F526275666665725F4E755A
:105A70006D203D202564200A00000000F047000052
:105A8000D0470000FA100000EC4C0000D04C0000A1
:105A9000EC2100000C4D0000F44C0000BE20000082
:105AA000384D0000204D0000BE2000005C4D00007D
:105AB000444D000052210000884D0000704D000050
:105AC00052210000B44D0000944D00000820000059
:105AD000E84D0000C84D000008200000104E0000F6
:105AE000F84D00004A1F00003C4E0000244E00000C
:105AF0004A1F0000644E00004C4E0000C81E00000B
:105B0000904E0000784E0000C81E0000B44E000009
:105B10009C4E00001C1E0000E04E0000C84E00001D
:105B20001C1E0000084F0000EC4E0000661D000027
:105B3000344F0000184F0000661D00004C4F00005D
:105B4000404F0000841C00006C4F0000604F0000BC
:105B5000841C00008C4F0000784F0000DA1B00000E
:105B6000AC4F0000984F0000DA1B0000C84F000047
:105B7000B44F0000C81B0000EC4F0000D84F0000DD
:105B8000C81B0000A0510000885100003622000010
:105B9000D0510000AC510000EC240000F85100008E
:105BA000DC510000DE240000A452000084520000FA
:105BB0003C2E0000C8520000AC520000222E000013
:105BC000EC520000D4520000082E0000D004000067
:105BD000D80400001C30000010360000DC04000077
:085BE0000C250000D4040000B4
:105BE80001000000040000200400002080000000E4
:105BF8000200000014000020140000202000000013
:105C080003000000240000202400002024000000DD
:105C180004000000340000203400002020000000B0
:105C2800050000004400002044000020300000006F
:105C3800060000005400002054000020340000003A
:105C480009000000640000206400002044000000F7
:105C58000A00000074000020740000202C000000DE
:105C6800FFFF00000000000000000000FFFF000030
:105C78000000000000000000FFFF0000000000001E
:105C880000000000FFFF000000000000000000000E
:105C9800FFFF00000000000000000000FFFF000000
:105CA8000000000000000000FFFF000000000000EE
:105CB80000000000FFFF00000000000000000000DE
:105CC800FFFF00000000000000000000FFFF0000D0
:105CD8000000000000000000FFFF000000000000BE
:105CE80000000000FFFF00000000000000000000AE
:105CF800FFFF00000000000000000000FFFF0000A0
:105D08000000000000000000FFFF0000000000008D
:105D180000000000FFFF000000000000000000007D
:105D28000000000000000000010203040607080943
:105D38000000000001020304010203040607080929
:085D480000D8B80502040608AA
:00000001FF
